:0600000002045B02020D88
:03000B000202618D
:030013000202F8EE
:01001B0032B2
:0100230032AA
:01002B0032A2
:0B045B0075811B120356E5826003024E
:02046600002C68
:080468007900E94400601B7AF1
:05047000009004D078AB
:0C0475000075A000E493F2A308B8000298
:0904810005A0D9F4DAF275A0FF20
:08048A007800E84400600C79E1
:0D04920000900000E4F0A3D8FCD9FAF6D8E1
:08049F00FDE4F509F508E4F5A0
:0504A7000DF50CE4F569
:0404AC000FF50E75C5
:0604B0001000751101753A
:0604B60012047513057528
:0604BC0014087515097516
:0604C200160C75170D7504
:0504C800180275190384
:0304CD0002002CFE
:05002C0012033380FE09
:0E003100C28C758C00758A00438901AA8974FF
:08003F00FD5AF589C28DD28C37
:010047002296
:040048007AFF7B00C0
:05004C001ABAFF011BC0
:04005100EA4B70F70F
:010055002288
:040056007A007B00B1
:0E005A00C374099A74808BF063F08095F050A7
:010068000493
:040069007A007B009E
:0D006D00EA2410F8860474704CF5907CFFB6
:02007A007D0007
:0E007C00C002C003C004C005120048D005D069
:0A008A0004D003D0021CBCFF011DCE
:04009400EC4D70E4DB
:050098000ABA00BE0BD6
:02009D0080BB26
:01009F00223E
:0D00A000AA82AB83EA2410F8860274704A2D
:0500AD00F590438702FD
:0100B200222B
:0600B300AA08AB09E4F508
:0C00B9001B751A648A828B83C002C0038E
:0D00C500120423AC82AD83D003D002E4F519
:0C00D2001B751A648C828D83C002C00371
:0E00DE00C004C00512035AAE82AF83D005D015
:0E00EC0004D003D002EAC39EFAEB9FFBE4F5BA
:0C00FA001B751A0A8A828B83C002C003A7
:0E010600C004C005120423AE82AF83D005D022
:0C01140004D003D002E4F51B751A0A8A1F
:0E012000828B83C004C005C006C0071203ED29
:0E012E00AB82A983D007D006D005D004EC2404
:0D013C0010F886028A04EA3395E0FDEE24F7
:0D01490010F886028A06EA3395E0FFEB24E9
:0D01560010F886028A03EA3395E0F98C90D8
:0E016300C003C004C006C007C001120048D08F
:0E01710001D007D006D004D003D296C003C040
:0E017F0004C006C007C001120048D001D0071E
:0E018D00D006D004D0038C90C003C006C0077B
:0E019B00C001120048D001D007D006D0038E5C
:0E01A900028A90C002C003C006C007C0011247
:0E01B7000048D001D007D006D003D00274203B
:0E01C5004EF590D295C002C003C00112004852
:0D01D300D001D003D0028A90C003C00112F9
:0E01E0000048D001D0038B028A90C002C003F9
:0E01EE00C001120048D001D003D00274104BA3
:0E01FC00F590D294C002120048D0028A9012F0
:02020A000048AA
:01020C0022CF
:0E020D00C0E0C0F0C082C083C002C003C004C5
:0E021B00C005C006C007C000C001C0D075D02D
:0C02290000C3E4950874808509F063F0C0
:050235008095F0500966
:08023A00150874FFB508021558
:0102420009B2
:030243001200B3F3
:0E024600D0D0D001D000D007D006D005D00413
:0D025400D003D002D083D082D0F0D0E032B1
:0E026100C0E0C0F0C082C083C002C003C00471
:0E026F00C005C006C007C000C001C0D075D0D9
:08027D0000050CE4B50C0205BC
:010285000D6B
:0302860030B34D45
:0C028900C3740F950C7480850DF063F0B9
:050295008095F05043CC
:08029A00E4F50DF50C30B33062
:0602A200E50A2508FAE55B
:0C02A8000B3509FBC374B49A74808BF012
:0702B40063F08095F0500893
:0802BB00E4F5097508B4800C9C
:0502C300E50A2508F525
:0402C80008E50B3505
:0302CC0009F50928
:0302CF001200B367
:0402D200C28C800753
:0702D600C28CE4F50DF50CEC
:0E02DD00D0D0D001D000D007D006D005D0047C
:0D02EB00D003D002D083D082D0F0D0E0321A
:0E02F800C0E0C0F0C082C083C002C003C004DA
:0E030600C005C006C007C000C001C0D075D041
:0403140000120031A2
:0E031800D0D0D001D000D007D006D005D00440
:0D032600D003D002D083D082D0F0D0E032DE
:09033300E4F580F5097508B41227
:0E033C0000B3D288D28AD2A8D2AAD2A9D2AF58
:06034A00E4F50B750A64E6
:0503500043870180FB62
:010355002285
:03035600758200AD
:010359002281
:0C035A00E582851AF0A4C582C0F0851B66
:0D036600F0A4D0F025F0C583851AF0A42581
:0403730083F5832269
:08037700E51A451B60467A01FE
:07037F00E51A25E0F51AE57F
:090386001B334012F51BE58295C2
:0A038F001AE583951B40030A80E67F
:03039900C3E51B9E
:07039C0013F51BE51A13F530
:0103A3001A3F
:0C03A400C3E582951AF5F0E583951B4037
:0603B00005F58385F082D3
:0703B600C3E51B13F51BE575
:0603BD001A13F51ADAE143
:0103C3002217
:0503C4007A10E4FBFCCF
:0E03C900E58225E0F582E58333F583EB33FB17
:0C03D700EC33FCEB951AF5F0EC951B40A4
:0703E30006FCABF0438201B0
:0303EA00DADD2237
:0E03ED00C2D5E58330E70DD2D5E4C39582F585
:0603FB0082E49583F58306
:0A040100E51B30E70BE4C3951AF584
:05040B001AE4951BF549
:010410001BD0
:0E04110012037730D50BE4C39582F582E49593
:03041F0083F583DF
:0104220022B7
:0E042300C2D5E58330E70DD2D5E4C39582F54E
:0604310082E49583F583CF
:0C043700E51B30E70DB2D5E4C3951AF5C3
:050443001AE4951BF511
:010448001B98
:0E0449001203C430D50BE4C39582F582E4950E
:0304570083F583A7
:01045A00227F
:00000001FF
